:030000000219FDE5
:03000B000200AA46
:03002B0002015C73
:03005B000202EEB0
:030073000202DBAB
:1000800002030406080C10182030406080040608A3
:100090000C10182030406080A0C00003070F1F0D17
:1000A0000D0403060D0503030202C2AFC0D0C0E079
:1000B000206214E5256009E473E525F4F58AD2622F
:1000C000D0E0D0D0D2AF3285268AC262E526F46075
:1000D0002F30682520720DD0E0D0D0D295D293D2A7
:1000E00097D2AF32D295D293D297206F0C20650968
:1000F0007406D5E0FDE57B4290D0E0D0D0D2AF329F
:10010000758A00C28DD26201F901B9306805206597
:1001100002C29501B9306805206502C29701B93065
:100120006805206502C29301B9C29430680A20654F
:10013000077406D5E0FDC29501B9C29630680A2061
:1001400065077406D5E0FDC29701B9C29230680A0E
:100150002065077406D5E0FDC29301B9C2AFC2ADF8
:1001600053E6EFC0D0C0E0D2D3D2AFC2CEE52A6012
:100170000720744F152A21C37800790020742EE5DA
:1001800080307E01F430E50278FF53DACF207E0321
:1001900043DA20307E0343DA10C2D8C271E58030E2
:1001A0007E01F430E50279FFC3E89970CB3061033A
:1001B000752A40207403752A40885CD270E8600379
:1001C000755F0020740DE52B6004152B21D343DAF5
:1001D00001C2D820700221E6A85C206102C2702012
:1001E000740221E488227882B6040385222420CF79
:1001F0000AD0E0D0D043E610D2AD32C2CF053A7873
:1002000002E52A6005307402152AC3E55C940140BA
:1002100005755F004127756000756900E55F240181
:10022000F55F5003755FFF7982B7020D306E1DC315
:10023000E52294324016854C227982B7030E306E47
:100240000BC3E52294324004798E8722C3E52395BF
:1002500022600840041523415B0523D8CA0569E5DF
:100260006970021569D56A69756A017808E56B607D
:10027000497805C3E569956B4057C3E569956C50AE
:10028000087801756A03020295C3E569956D50050A
:100290007801756A01C3E5629524401E7982B7042E
:1002A0000241C6206E14852462E569046003856BF3
:1002B00069756A0175233C0202D1E5622850057513
:1002C00062FF41C6F562E5620470067560FF7569FC
:1002D000FFD0E0D0D043E610D2AD32C2AF53E67FBC
:1002E0007592FA7593FFC260759104D2AF32C2AFB6
:1002F00053E6EFC2ADC0D0C0E0C0F0D2D3D2AFA8B9
:10030000FBA9FCC2D8307102615553DACF207E03BD
:1003100043DA10307E0343DA20D271E580307E016B
:10032000F420E502612C88278928A13A53DACF20EE
:100330007E0343DA20307E0343DA10C2D8C2713024
:100340007402A1267800E580307E01F430E502A138
:1003500026885CA10E53DACF207E0343DA20307E5C
:100360000343DA10C271206102812E53DACF207E5E
:100370000343DA10307E0343DA20C2D8D2718857A3
:100380008958C3E89555F8E99556F97B007E087AB7
:1003900000C3E8948CE994005005755B00812088C7
:1003A0002178A2E6A8216055C3E894C8E9940050DA
:1003B00008E4D2E4FB7A0A61FBC3E89468E994019B
:1003C0005008E4D2E3FB7A0F61FBC3E894D0E994D0
:1003D000025008E4D2E2FB7A1E61FBC3E894A0E974
:1003E00094055008E4D2E1FB7A3C61FBC3E89498A1
:1003F000E994085008E4D2E0FB7A787E00C3E895DF
:1004000059FCE9955AFD30E70AECF42401FCEDF4BF
:100410003400FD755B00C3EC9AED9E5003755B01E3
:100420008859895A8557558558567802A10EC3E8D0
:100430009527F8E99528F9307C0281F2307B02811A
:10044000F2307A0281EB2075028151E9FDE8FC81EE
:1004500070E9C313F9E813F830790281EBE9C313AB
:10046000F9E813F830780281EBE9C313FDE813FCD7
:0F04700020612CC3EC941CED940240028187EDB7
:10047F00701EC3EC94C850180529E5297002152980
:10048F00C3E529940A5002A126755C00D270A126FB
:10049F00E529600215297400207F037896E624FA77
:1004AF00FEE43400FFC3EC9EFCED9FFD5006780088
:1004BF00790081F2C3EC94FFED9400400678FF7948
:1004CF000081F2EC8572F0A4C5F0A2F733F8790041
:1004DF00400302050E78FF790002050EE9C313F9F8
:1004EF00E813F8307C0EE9600278FFC3E81338F8A0
:1004FF00E43400F9C3E894FFE99400400278FF88E0
:10050F005CD270206102A126741FF4552F4BF52F7A
:10051F00C274EB7002D274752A40307403752A0AC4
:10052F00306102A13A20740353DAFE207403752B55
:10053F0020D0F0D0E0D0D0D2AD43E6103279010216
:10054F00056A790302056A790A02056A791E0205AE
:10055F006A796402056A79C802056A7817E4D5E0FA
:10056F00FDD8FAD9F6227A147B780205917A107B9E
:10057F008C0205917A0D7BB40205917A0B7BC80230
:10058F000591E573D5E001227902E4C296D5E0FD2D
:10059F00C297D5E0FDD297D5E0FDD296D5E0FDE923
:1005AF0020E002C29530E002C293E573D5E0FDE989
:1005BF0020E002D29530E002D2937496D5E0FDD9B7
:1005CF00C9EAF8D5E0FDD8FBDBB8C29622C37C00A0
:1005DF007D0075F00005F0EA33FAEB33FB50F6EBD4
:1005EF0013FBEA13FAC3E9FFE8FEE89AF8E99BF96F
:1005FF005004EFF9EEF8B3EC33FCED33FDD5F0DF3B
:10060F00EDF9ECF822E889F08A20D2D4F8A9F07B32
:10061F000030F70B7BFFF42401F8E9F43400F9E81C
:10062F008520F0A4ADF0F8E98520F0A4AFF0FEED41
:10063F002EF974003FFA7C04C3EA13FAE913F9E8C0
:10064F0013F8DCF48BF030F70AE8F42401F8E9F43E
:10065F003400F9E889F0C2D4F8A9F0227882B60400
:10066F000302070AC3E55C9419401EE52D5406707A
:10067F0018206E3678057994E7146007780A1460AD
:10068F00027812C3E54198401F306E098564627588
:10069F0069FF756A01852224E4F544F545F546F5B1
:1006AF0047F548C26E02070AD26E7994E7147013A9
:1006BF00E523F43333F913F8E9540104F9E854FE50
:1006CF000206FEE714147014E523F4333333F913E1
:1006DF00F8E9540304F9E854FC020706E523F43360
:1006EF00333333F913F8E954070404F9E854F8C322
:1006FF009440F8E99400F98844894522C3E54113F1
:10070F00F9E54013F8C3E54498F8E54599F9500C1D
:10071F00C3E89480E994FF4016020742C3E8947F30
:10072F00E994005003020742787F7900020742786C
:10073F008079FF8849894A22E5492546F8E54A35F7
:10074F0047F9854A20E4300701F43548FA30E709C4
:10075F00C3EA94F04015020780C3EA940F500302D6
:10076F00078078FF79FF7A0F020780780079007A87
:10077F00F0C3E5249561500AC374019524500B0210
:10078F00079EE54A20E70E02079EE54A30E70688F6
:10079F004689478A482278A5E6FAC3E54933F8E542
:1007AF004A33F9D114E930E70BC3E89480E994FF99
:1007BF004013E1D8C3E8947FE994005002E1D87860
:1007CF007F7900E1D8788079FFE820E715C3E5232A
:1007DF0098F84009C3E8940140030207FF7801022B
:1007EF0007FFE8F424012523F840030207FF78FFF1
:1007FF00884B2278A6E6FAA847A948120614E930D2
:10080F00E70CC3E89401E994FF4016020834C3E8EB
:10081F0094FFE99400500302083478FF790002082E
:10082F0034780179FFE920E715C3E54B98F84009C3
:10083F00C3E89401400302085B780102085BE8F407
:10084F002401254BF8400302085B78FF88242278A7
:10085F00FF20692879A1E76023E541601F74FF85B8
:0E086F0041F0848539F0306A0375F005A4F875
:10087D00C5F0600278FFC3E895645002A8648863F0
:10088D0022C3E5409440E5419401E5635003140112
:10089D009F046002F563227883E6F520120F21751F
:1008AD00E89012054C75E89030EDFDA8BDA9BE127B
:1008BD000FC8756E55756F00C3740013FD745560C8
:1008CD006613FC74552CFC74003DFDECFAEDFBC376
:1008DD00E89AE99B4014E56E2455F56EE56F3400FA
:1008ED00F56FEA2CFAEB3DFB80E5AE6EAF6FC3E51D
:1008FD006F13F9E56E13F8C3E913F9E813F87A03EA
:10090D00C3E913F9E813F8DAF7AA201A7009756E1E
:10091D0000756F000209341AEA6008EE28FEEF39FF
:10092D00FFDAF88E6E8F6F2275E890227883E6FFDE
:10093D0030EDF9A8BDA9BE0570C3E570940840520D
:10094D00757000E9FA79A0E76044EA7007E5716017
:10095D001B02096DC3E895716010E5715006600CBE
:10096D00140209790460F9020979E571F571C394EE
:10097D006D401B7561C0C394044013756180C394B1
:10098D0004400B756140C39404400375610075BB51
:10099D000822EFC39401601F7455601BC3E894FFD8
:1009AD00E994035012C3E8956EE9956F5009E5611E
:1009BD00600C15610209CBE561F460020561A86167
:1009CD00C3E524985002A824C3E89562400AA862A2
:1009DD00E562F4600385626188258826E570B407B9
:1009ED000375BB1022743279A787F0A4C5F0A2F766
:1009FD0033F8C3E895614002A861882288248825D0
:100A0D0088268864227540007541F022C2AF75C8F2
:100A1D0020A8CCA9CDAA3A30CF010A75C824D2AFEF
:100A2D00AB3BAC3C883B893CC3E89BF8E99C206917
:100A3D0008F9306602612A4184AD3D8A3DF9EA9D8F
:100A4D00FA600678FF79FF4169AE3EAF3F8B3E8C71
:100A5D003FA83BA93CC3E89EF8E99FF9C3E54113C4
:100A6D00FBE54013FAE82AF540E93BF541500675E0
:100A7D0040FF7541FF41D1AA40AB41AC40AD417E35
:100A8D00047F02C3EB9404400D1E1FC3EB9408407A
:100A9D0005206A021E1FC3ED13FDEC13FCDEF7C328
:100AAD00EA9CFAEB9DFBEF6009C3E913F9E813F833
:100ABD00DFF7EA28FAEB39FB8A408B4150067BFFC2
:100ACD008B408B41C3EB94025002D2663069047F98
:100ADD000341FC7892E6FFC3E537948240110FC3C2
:100AED00E53794A040010FC3EF940640027F057EC9
:100AFD0002E541C4540FF9E541C454F0F8E540C492
:100B0D00540F28F8C3E89EFAE99400FB4009C3EAA4
:100B1D009402EB940050047A02E4FB6176AA40AB98
:100B2D0041EBC4FEEAC4540F4EFCC3EA9CFAEB94AD
:100B3D0000FBC3E813C313F8EA28FAEB3400FB8A71
:100B4D00408B41C3EB94024002C2667802EBC4FEB7
:100B5D007B00EAC4540F4EFAC3EA98FA4005C394D9
:100B6D000250027A027892E6FF306002617685517A
:100B7D0092855293D26043E680C3E49AF8E49BF9E0
:100B8D003066028102E8FAE9FBD3E913FDE813FCB4
:100B9D0088518952C3EF94036038EF20E00DE82CA3
:100BAD00F8E93DF9ECFAEDFB020BCBE828F8E93951
:100BBD00F9C3E82402F8E93400F97AFE7BFFC3EFAC
:100BCD009403400E8A538B54884D894E8C4F8D5013
:100BDD008136885389548A4D8B4E8C4F8D50306998
:100BED00127553F07554FF754FF07550FF7551F038
:100BFD007552FF8136E8FAD3E813FC8851C3EF94A0
:100C0D00036020EF20E007E82CF8ECFA8122E828B9
:100C1D002402F87AFEC3EF940340088A53884D8C62
:100C2D004F813688538A4D8C4FE568C3335002642B
:100C3D006BF5683060028140753402D26043E68006
:100C4D00E52D54066034A840A941C3E913F9E81312
:100C5D00F8C3E913F9E813F8306904E92440F9C23F
:0E0C6D00AF53E67F759100C3E498F594E499C7
:100C7B00F595759104D26043E680D2AF22D26475AC
:100C8B004300752000306C03752040020CA7D26422
:100C9B00754300752040306C037520007801790195
:100CAB00206620E52D54066002C2647914E541C329
:100CBB0013700104F8C3941440027814306904785B
:100CCB001B791B206010E543600C306903D534049D
:100CDB00D26DA15191480543E59B5440B52002A12B
:100CEB003B30690908C3E89940011881CE20640A9A
:100CFB0008C3E899400281A781CEC264C2AF53E614
:100D0B007F7591003066127594007595F875910496
:100D1B00D26043E680D2AF81A7E5417EFFC333406B
:100D2B0005C3334001FEC3E49E759400F595A118ED
:100D3B00C3E5339401500281A730640281A7D80226
:100D4B00A14F81CEC26DC2AF53E67F759100855323
:100D5B0094855495759104854D92854E93D260433D
:100D6B00E680D2AFE52D54066008206A02053302F7
:100D7B000D8D306D0D206C0A2064071581158102D5
:100D8B0016362278003064027801E53775F007A437
:100D9B00F9E5F028F5F0E9A2F013A2F113A2F21392
:100DAB00F537C394785003753778C3E537953840DA
:100DBB0008D265D295D293D297306002A1C4854FE9
:100DCB0092855093D26043E68022207D16C2AF7588
:100DDB004202C296D294306202C293D2AF759F1177
:100DEB00020FC5C2AF754202C296D292306202C2E6
:100DFB0095D2AF759F11020FC5307243207D20C273
:100E0B00AF75420390013A757B40D293C292306228
:100E1B0004C297C122D296D2AF759F13020FC5C2DF
:100E2B00AF75420390013A757B40D295C294306204
:100E3B0004C297C142D296D2AF759F10020FC52044
:100E4B007D17C2AF754203900115D293306202C277
:100E5B0097D2AF759F13020FC5C2AF7542039001B6
:100E6B0015D295306202C297D2AF759F10020FC593
:100E7B00207D16C2AF754204C294D292306202C278
:100E8B0097D2AF759F10020FC5C2AF754204C292C5
:100E9B00D294306202C297D2AF759F13020FC53046
:100EAB007243207D20C2AF754205900129757B10DE
:100EBB00D297C296306204C295C1C8D294D2AF7594
:100ECB009F11020FC5C2AF75420590014B757B0494
:100EDB00D297C296306204C293C1E8D292D2AF7558
:100EEB009F11020FC5207D17C2AF75420590010BF4
:100EFB00D297306202C295D2AF759F11020FC5C255
:100F0B00AF75420590011FD2973062EBC293D2AFFF
:100F1B00759F11020FC5207D16C2AF754206C29296
:100F2B00D296306202C295D2AF759F13020FC5C223
:100F3B00AF754206C294D296306202C293D2AF759D
:100F4B009F10020FC5307244207D20C2AF75420145
:100F5B0090014B757B04D295C294306204C293E12D
:100F6B006ED292D2AF759F10020FC5C2AF75420100
:100F7B00900129757B10D293C292306205C2950203
:100F8B000F8FD294D2AF759F13020FC5207D17C25E
:100F9B00AF75420190011FD295306202C293D2AF5E
:100FAB00759F10020FC5C2AF75420190010BD29312
:100FBB00306202C295D2AF759F13C26522900109B0
:100FCB00757B00D295D293D297C294C292C296C22D
:100FDB00622278807607087607087601087604087F
:100FEB0076FF0876FF08760A0876020876010876FF
:100FFB0001788C76010876000876B40876FF0876BF
:10100B00FF0876FF0876030876FF0876010876FF5F
:10101B000876250876D00876780876C8087604080E
:10102B0076FF08760108760008767A08760A087645
:10103B00010876010876000876FF0876002278878B
:10104B00E6FFC272BF0302D2727888C27DE630E13E
:10105B0002D27DC27E7889E630E102D27EC3EF9464
:0E106B00026008758E01D27302107B758E0034
:10107900C273227880E6149000809378A5F678816F
:10108900E6149000809378A6F67886E61490008D91
:101099009378A7F6789FE6F87005756B0001C2C3CF
:1010A900E8941140027811E82828F56B256B256B27
:1010B90028F56C256B2828F56D7886E6F539C394F3
:1010C900025003753902789CE67538FFB40203753E
:1010D90038A0B4030375388278A3E61490009A9374
:1010E900F566120FC822227896E6FA7897E6FB7819
:1010F90088E6B40305C3EB940EFB307F047A007BCA
:10110900FFC3EB9AFCC3948250027C82757200057E
:1011190072EC8572F0A4C3E5F0947D40F222D27F8F
:1011290011F012055B12055B7A007B007C10120539
:1011390051E55C2AFA74003BFBDCF37C04C3EB1336
:10114900FBEA13FADCF7FEC27F11F022757C007509
:101159007D00E5EF20E6037520000520903FFFE5BF
:1011690020146006901DFF1460009304600375EF5E
:101179001653D9BF7581C043FF8012054C75EF0620
:1011890043B203E5B3240220E70DF521E5E320E0AE
:10119900068521B343E301120FC87580FF75A400CA
:1011A90075F1B275D4DF7590A975A5FC75F2FE7558
:1011B900D50175A60175E241120FC8E4F8F6D8FD0C
:1011C900756801120FDD12168D78988673753001D6
:1011D900C2AF12056512057512055B12057C120571
:1011E9005B12058312055B1217C0120565120565AE
:1011F900120560C2AF757C00757D0078FA79FA3006
:101209008507D9FBD8F7021C001149117C11EF1190
:10121900F078988673120FC875881075890275C899
:101229002475910475D84075A82275B80275E690A1
:10123900759B80759D0075D10E75BC5875BB087579
:10124900BA1175E88012054CD2AF1208A4753600A0
:1012590053DACF207E0343DA20307E0343DA10438A
:10126900DA01C2D8C271120565D2617B037A0CE535
:101279005B70077A0CDB030211FC12055B2070031B
:101289000211FCC270E55CC3940240E1E52F541FD2
:10129900855E5DF55EB55DD5DAD5C26153DACF20DD
:1012A9007E0343DA20307E0343DA10C2D8C2717854
:1012B900A2E67008D274E52F54E0F52FC27575299E
:1012C90000120560307409C3E529940A4002D275F9
:1012D90012055178023074027800C3E55C9840F039
:1012E900C2AF120575120575120575D2AF120565E3
:1012F900754C00120551788CE6C394015003021312
:10130900E9E530C3940150030213E9757CA5757DA5
:10131900F1207435C3E55C94FF50030213E9C2AFB1
:1013290012058AD2AF120560C3E55C940150EFC281
:10133900AF120575120556120575D2AF120560C3B5
:10134900E55C94FF40E90218457F05D27F11F01250
:101359000560C2AFC27F11F0AE5CC3E55C947FD279
:10136900AF500261F912054CC2AF12058AD2AFDF44
:10137900DA3127C3EE94057897F61205651217C876
:101389007F0AD27F11F0120560C2AFC27F11F0AEA1
:101399005CC3E55C947FD2AF50E612054CC2AF1234
:1013A9000575120556120575D2AFDFD63127EE2421
:1013B900037896F6F87997E7C39482400398500624
:1013C900E824827897F61205651216DB1217F712D0
:1013D900056011F0C3E55C94FF50026114021845E1
:1013E900757C00757D00C3E55C954C4003855C4CBC
:1013F90012056078017988E7B403027805C3E55CD2
:1014090098400241FCC2AF12058A12058A12058A68
:10141900D2AF120565753000E4F531F5320531E5D5
:1014290031F4703F0532789AE678191460127832EF
:1014390014600D787D14600878FA14600375320021
:10144900C3E53298401D120FC812054C153275318B
:101459000078998673C2AF12058AD2AF78988673DD
:0F146900120560120556E52A700530740221FC49
:1014780078012074027806C3E55C9840A1120560E3
:10148800E52A70030211FCC2AF120FC8E4F522F579
:1014980023F524F525F526F567D2AF7885E6C3331D
:1014A800F565E4F544F545F546F547F548F570F575
:1014B8002CF52DF53775700875BB1012054C1209FF
:1014C8003530EDFDA8BDA9BEE97001F88871120993
:1014D8003975700875BB101149C2AF7561FF1209E3
:1014E800F2852261852262852263D2AF7522017559
:1014F8002401752501752601856069756A0178885A
:10150800E6B40307C27D307602D27DD268D269750F
:101518003300120F21120F50120A12120A19120A5E
:1015280012120A19120A12120C9912066B120D8E57
:10153800120DD5120A19120C88306E0312070B20EF
:10154800660312085E30660312088E120D8E120EA4
:1015580004120A19120C99306E03120747120D8EE5
:10156800120E7B120A19120C88306E031207A5128C
:101578000D8E120EAA120A19120C99306E03120857
:1015880002120D8E120F21120A19120935120C8837
:10159800120D8E120F50120939120A1930692C8552
:1015A8006461856462856069756A0179187A0CC31B
:1015B800E533994009C269D26A8A350215D3C3E571
:1015C8005C9401400302152F02163E306A25206CF8
:1015D80022E535147006C26AD26BA12FF535C3E532
:1015E8005C9401400302152F7888E6C394036003D6
:1015F80002163E753600C3E55F94014009856462B2
:10160800856069756A0178FA79A4E760027803C38E
:10161800E55F985021307404E52A601A78F0306C40
:10162800058564617820C3E541985002A12F0536ED
:10163800E55C6002C141753600C2AF120FC87887F9
:10164800E6FE760211497887EEF6E4F522F523F5F1
:1016580024F525F526F565752C00752D00D2AF12F9
:101668000560120FC878A4E66006C295C297C293B7
:10167800307406E52A700221FC788DE6C394014097
:101688000241D98121901A0D782012171DE520B446
:10169800A50CA312171DE520B45A030216BB757CCE
:1016A800A5757DF1120FDD1216DB757C00757D00C6
:1016B8000216DA901A0378807B0A12171DA308DB3A
:1016C800F9901A0F788C7B1912171DA308DBF99073
:1016D8001A2822C2AF12176012173D901A00740E12
:1016E800121722A37409121722A374151217229035
:1016F8001A0378807B0A121721A308DBF9901A0FC6
:10170800788C7B19121721A308DBF91217731217AB
:1017180051901A2822E493F622E6438F01538FFD55
:10172800FFC3E583941C400122EF857CB7857DB714
:10173800F0538FFE22438F02438F01857CB7857D4E
:10174800B7901A0DF0538FFC22901A0D74A5F12250
:10175800901A0E745AF122227A3079D07820901A91
:1017680040F11DE520F709A3DAF7227A3079D09005
:101778001A40E7F12209A3DAF922AB74A875BB0174
:10178800027980BB02027981BB03027982BB040221
:101798007994BB05027983BB06027986BB07027977
:1017A80092BB08027987BB0902799CBB0A02798837
:1017B800BB0B027989E8F7227C05120565DCFB2260
:1017C800C2AF12057512057C12058312058A12052F
:1017D8005612057512057C12058312058A120556E4
:1017E80012057512057C12058312058AD2AF22C232
:1017F800AF12058A12058312057C1205751205566B
:1018080012058A12058312057C12057512055612F7
:10181800058A12058312057C120575D2AF22AE74B3
:10182800AF75C2AF1205751205751205751205560A
:10183800DEF212058A120556DFF8D2AF221217C857
:101848001217C01217C075740175750175760011ED
:10185800267C05AD5C120565C3ED955C70F5C3E5A6
:0F1868005C9401400AC3E55C94FF403702188886
:101877001217821216DB1217C8C2AF75EF161217AE
:10188700C0DCD10576C3E5769403500280C21217F7
:10189700C00575E5741490009F93F808C3E5759823
:1018A700500280A91217C01217C00574C3E57494BB
:1018B7000C50028095120FDD1216DBC2AF75EF16C2
:0318C7001217C035
:0319FD000211557F
:101A00000E091507070104FFFF0A020101A55A018B
:101A100000B4FFFFFF03FF01FF25D078C804FF01DA
:091A200000FF0A010100FF00FFB4
:101A4000235475726E6967794E6665743235412329
:101A500023424C48454C4923463333302320202031
:101A60002020202020202020202020202020202076
:101C0000C2AFC2D353D9BF7581C043B20343FF8073
:101C1000752438752503B1DC7529A5752AF175E29F
:101C20004043F12053A4DF75D4FFD2857DFA7803B9
:101C300079E67C10752200752300901DE97B0675FE
:101C400024987525013085028145208508D8FBD967
:101C5000F9DCF781B7308508D8FBD9F9DCF781B713
:101C6000B19CE493A3C39A6004DDC381B7DBDBB10D
:101C70008E6002812E7B08E493FAA3B16FDBF87AC1
:101C800030B16F752200752300B18EEAFCEBFDC305
:101C9000ED94FE400EB18E8A278B28ED30E0048A49
:101CA000828B83B18E7AC270D8C3ED94FE601950D6
:101CB000CEBD002BEC600F7520007521FF7529004B
:101CC000752A000200008100A827A9280809D80465
:101CD000D90281DCB192EA89AAF281CE0D81A3C337
:101CE000ED94035053EDA2E092007AC5C3E58294CF
:101CF00000E583941C508A200010438F02438F011B
:101D00008529B7852AB7F0300029A827A92808090E
:101D1000438F01538FFDD804D902A133C3E58394C7
:101D20001C4003A3A11689AAE28529B7852AB7F02A
:101D3000A3A116538FFC817F7AC1BD030CE493A34A
:101D4000FAB153DCF8B14B817F8181AA22AB23B178
:101D50006FEBFAEA6222752608C3E52313F523E543
:101D60002213F52250066323A0632201D526EAB18F
:101D7000DCB1DC75260AEAF4200102D285300102CA
:101D8000C285B1DCC3134002C201D526EB22B19259
:101D9000EAFB208502A192308502A197752608AE44
:101DA00024AF25C3EF13FFEE13FEB1E0B1DCC3EAAD
:101DB000133085024480FA30E703632201C3E52330
:101DC00013F523E52213F52250066323A0632201B5
:101DD000D526D9E52265236523F52222AE24AF2539
:101DE0000E0FDEFEDFFCD20122424C48656C6934E6
:071DF000373164F3300601F6
:00000001FF
